S018000064656D6F70726F675F7333326B3131382E7372656373
S1132000005800202D2E0000FB2A0000FB2A0000AF
S113201000000000000000000000000000000000BC
S1132020000000000000000000000000FB2A000087
S11320300000000000000000FB2A0000292B000023
S1132040FB2A0000FB2A0000FB2A0000FB2A0000F8
S1132050FB2A0000FB2A0000FB2A0000FB2A0000E8
S1132060FB2A0000FB2A0000FB2A0000FB2A0000D8
S1132070FB2A0000FB2A0000FB2A0000FB2A0000C8
S1132080FB2A0000FB2A0000FB2A0000FB2A0000B8
S1132090FB2A0000FB2A0000FB2A0000FB2A0000A8
S11320A0FB2A0000FB2A0000FB2A0000FB2A000098
S11320B0FB2A0000FB2A0000FB2A0000FB2A000088
S10720C0EE11AA551A
S1132400FFFFFFFFFFFFFFFFFFFFFFFFFE7FFFFF59
S113241080B500F00DF800F087F901BD80B500F03B
S113242059F800F04BFA01BD80B500F0E9FA01BD9E
S11324301CB568469B490CC90CC0083908389A4831
S11324400168A54A0A40026001688422D2050A4351
S11324500260A2480168090A4907490F002905D109
S113246001210A02E023DB00134003609C4801249D
S11324709C4A12682240002A00D19B486A46515C5B
S113248000F0E4FAE121090200F0E0FAC01DC008FE
S1132490C004C00C80B2C004C00CE021C9040143D4
S11324A09248016092489349086093480021016072
S11324B0924A1160924A11609249F02292020A6093
S11324C00A68882313430B608F490C60C0210903F9
S11324D0016013BD70B58D4C2078002815D18C4D4A
S11324E0280000F037F8012833D12878002830D0AC
S11324F0287841282DDA00F014FB86490860012071
S1132500207000208449087023E0834D804E287891
S11325103018401C00F01EF8012811D12878401C06
S1132520287028783178884213D100202070707880
S1132530FF280ED1B07800280BD1FFF775FF08E013
S113254000F0EFFA734909686431814201D2002036
S1132550207070BD00B500210122664B1B685B0D25
S11325601340002B03D0D3490968017011000800FF
S1132570C0B200BDFEB507000D00140068466749EF
S11325800CC90CC00839083865480168090A4907AC
S1132590490F002905D101210A02E023DB00134081
S11325A0036060486A46515C00F050FA01900026CE
S11325B06846078000E0761C3000C0B212282BD297
S11325C0BD4F019869460A883100C9B204235943B2
S11325D0795C514300F03AFA0029ECD1019869463C
S11325E00A883100C9B204235943795C514300F08D
S11325F02DFA288028880028DDD02888FF21891C0E
S11326008842D8D22000F6B204214E43B9190422DC
S113261000F0B4FA012000E00020FEBD38B5C24C41
S113262020688021C9050143216020688021490573
S11326300143216000F075FA0500FA352068C001F5
S113264003D400F06EFA8542F8D231BD38B5B64CE9
S113265020682149014021602068B449014021607B
S113266000F05FFA0500FA352068C00103D500F0D8
S113267058FA8542F8D231BD38B5AB4C20680028F1
S11326800FD42068802109060143216000F049FA33
S11326900500FA352068C00203D400F042FA8542EE
S11326A0F8D231BD242F0000A851064038B59E4C05
S11326B0206800280ED5206840004008206000F003
S11326C030FA0500FA352068C00203D500F029FA73
S11326D08542F8D231BD0000FFFFFFBF044206402F
S11326E000127A000842064080841E0010A00640B2
S11326F000C01FC014A0064018A0064020A0064039
S113270024A0064028A006402CA006401531002035
S1132710C030002004310020143100202C2F000090
S113272004410640409C0000FEB50027380069467D
S113273008800422002101A800F02DFA7C4D7D4878
S113274001688022D2050A430260FFF7AFFFFFF75A
S113275065FFFFF791FF784C2068784901402160BC
S1132760FFF7A4FFFFF75AFF01AA6946FA204000C9
S1132770FFF700FF20687249014021602068694624
S11327800988491E09060143216001A8216842788D
S1132790521E5207520F0A43226021688278521E49
S11327A0D204E0239B0313400B4323602168C278C7
S11327B0521E1204E023DB0213400B432360817892
S11327C0042901DA807800E004202168C0B2401EA8
S11327D08005C022120402400A432260206880213E
S11327E001432160380006E05649020092B20423F6
S11327F05343CF50401C010089B28029F4D33800E0
S113280006E05149020092B204235343CF50401CC6
S1132810010089B22029F4D3434E30687F218843D4
S11328201F210143316030688021890201433160F6
S113283030688021490201433160306843490140D6
S1132840316043484349086043488021C90401601A
S1132850002D0BD569004908026880239B031343AC
S11328600360C800C0083D49086004E0A804C00033
S1132870C0083A4908603A4807600020C043394913
S11328800860394839490860306839490140316085
S11328902068384901402160FFF7D8FE00F041F973
S11328A00400FA343068000103D500F03AF9844298
S11328B0F8D2F7BD1CA00640842E0000FEB580208F
S11328C0800028490A680240002A2BD0224A126854
S11328D0120C1207120F284B00240FE02500EDB252
S11328E00326B543ED1C2600F6B2B607B60FAD1BA2
S11328F05D5D6E462700FFB2F555641C2500160089
S1132900EDB2F6B2B542E9D308601C4800681C4930
S1132910086068460078FF2804D1D2B2022A01D1A7
S1132920FFF782FDF7BD000000400240FFFFFFEF0C
S1132930670600009050064004400240FFDFFFFF9E
S113294078FF00008040024080480240FFFFFFDF24
S1132950FFFFFF5FA44802401041024014410240BF
S1132960284002403040024006003B002040024024
S1132970FFFF7FFFF7EFFFFF1841024008400240CE
S11329800831002023482449016000682348244971
S11329900860244824490860704770B5002210007C
S11329A001252B000F24214E3168090C2140491CBC
S11329B03668360E3440012C04D018D3032C0CD0C6
S11329C002D314E01A4813E01A4C24682540002D61
S11329D001D0174800E013000AE0174C2468A4074C
S11329E0A40F002C01D1154800E0130000E01300EF
S11329F0DBB2002B03D000F029F81149086070BD48
S1132A00104A106880B21049014304200843106042
S1132A10704700000420054020C528D9202100006B
S1132A2000200540FFFF000008200540104006403C
S1132A3000127A000842064008430640006CDC029B
S1132A40C00000200CED00E00000FA050022030A9B
S1132A508B420BD203098B4219D243088B422ED2EC
S1132A60411A00D20146524110467047FF22090222
S1132A703FD012068B4205D3121209028B4201D3B6
S1132A801212090203098B4219D300E0090AC3098F
S1132A908B4201D3CB01C01A524183098B4201D32B
S1132AA08B01C01A524143098B4201D34B01C01A16
S1132AB0524103098B4201D30B01C01A5241C3088E
S1132AC08B4201D3CB00C01A524183088B4201D3FD
S1132AD08B00C01A524143088B4201D34B00C01AE9
S1132AE05241884200D3401A5241CFD20146104687
S1132AF0704708B500F05AF808BDFEE700B50D4868
S1132B000068FA218900FFF7A1FF401E0A49086006
S1132B1000200A4908600721094A11600949086030
S1132B2000BD08480068704706480168491C0160F8
S1132B3070470000C000002014E000E018E000E04E
S1132B4010E000E01031002070B4103A03D378C9CB
S1132B50103A78C0FBD2530701D318C918C001D565
S1132B6008C908C0D20704D30B880380891C801CC1
S1132B70002A01D50B78037070BC70478B0701D114
S1132B808307E1D0124205D00B78491C0370401C26
S1132B90521EF9D1704710B504000800110002005C
S1132BA0200000F005F8200010BD00007047000070
S1132BB01206130A1A43130C1A4300BF094205D024
S1132BC0830705D00270401C491EF9D170470000EC
S1132BD01300103906D330B41400150010393CC06A
S1132BE0FCD230BC490700D30CC000D504C0890016
S1132BF002D30280801C002900D5027070470000B7
S1132C0080B500F007F8FFF703FC00F076F8FFF753
S1132C1005FCFAE780B500F024F88020C0052249BD
S1132C200A6802430A6021490A6810430860802048
S1132C3080001F490A6802430A601E490A6810435B
S1132C400860A020C0001C490A6802430A601B49AE
S1132C500A6810430860FFF751FF00F041F862B6BC
S1132C6001BD80B5FF20801C154908603421154A38
S1132C70116015490A681202FBD401220A600A682D
S1132C80D201FCD511490860114908601148124964
S1132C90086012480068000E0007000F0328F8D1EE
S1132CA0FFF77BFE01BD0000285106403451064069
S1132CB000A0044004A0044010D0044014D00440F8
S1132CC004410640084106400041064004430640D2
S1132CD00442064001000003144006401040064030
S1132CE0802040001549086015490A6802430A60BB
S1132CF014490A6810430860704710B5FFF711FFC4
S1132D0011490A68821AFA235B009A4215D30F4AC2
S1132D101378002B08D1012313700D4A1368802403
S1132D2064001C43146007E000231370054A136811
S1132D30802464001C431460086010BD20D004404B
S1132D4014F10F4008F10F400C310020163100201F
S1132D5004F10F40FFB526482649274A0392274A23
S1132D60274B284C0294284C284D0195284D294E78
S1132D70294F009703E00F780770401C491C039FFC
S1132D808F42F8D10298984207D018781070521CDC
S1132D905B1CF7E700202070641C0198A042F9D165
S1132DA00098B04204D030782870761C6D1CF7E788
S1132DB00023180019491A4A8A4212D006E0042452
S1132DC05C430C5904255D4354515B1C154CA40809
S1132DD0A342F4D31449C0B20423584308580260F0
S1132DE005E0114AC0B20423584310580160FFBDE6
S1132DF0C0000020382F00003C2F0000C400002039
S1132E003C2F00003C2F0000C03000201731002070
S1132E10000000000000000000000000002000008E
S1132E2000000020C0000000342F000072B6002112
S1132E30002200230024002500260027B846B946B6
S1132E40BA46BB46BC460A490A4A521A013A05DD4B
S1132E500020042308601944043AFBDA0648854636
S1132E60064880470648804762B6FFF7C9FEFEE77A
S1132E7000000020FF570020005800208529000092
S1132E80552D000008030202090303020A03030389
S1132E900B0403030C0404030D0504030E050404CE
S1132EA00F0604041006050411070504120705059E
S1132EB0130805051408060515080705160807066E
S1132EC017080806180808071908080800F00DF87C
S1132ED0002801D000BF00BF00BF00BF002000BF1A
S1132EE000BFFFF78DFE00F002F80120704780B5A7
S1132EF000F002F801BD00000746384600F002F871
S1132F00FBE7000080B500BF00BF024A1100182093
S1132F10ABBEFBE72600020000BF00BF00BF00BF3E
S1132F20FFF7D4FF0001020408102040000102044E
S10F2F300810204008ED00E0006CDC02FA
S9032F19B4
